:0500000002003361D98C
:02000B0061DAB8
:02001300813A30
:02001B00813B27
:02002300813C1E
:02002B00813D15
:10003300759840758780758921758DFF758BFF7560
:100043008850D29975816075A8827530007531002A
:10005300D214D215D216D217D218D219D21AD21B51
:10006300D21CD21DD21ED21FD220D221D222D22301
:10007300D224D225D226D227D228D229D22AD22BB1
:10008300D22CD22DD22ED22FD234D235D236D23751
:10009300D250C251C291D292209214301421C21470
:1000A300B21520150512044C801512048880102007
:1000B300140DD21420150512046A80031204A6D26B
:1000C30091D293209314301621C216B2172017052C
:1000D3001204C48015120500801020160DD21620BC
:1000E30017051204E2800312051ED29420941430E3
:1000F3001821C218B21920190512053C80151205E2
:1001030078801020180DD21820190512055A800383
:10011300120596D295209514301A21C21AB21B20CB
:100123001B051205B480151205F08010201A0DD29C
:100133001A201B051205D2800312060ED2962096B2
:1001430014301C21C21CB21D201D0512062C801563
:100153001206688010201C0DD21C201D0512064AB1
:100163008003120686D297209714301E21C21EB236
:100173001F201F051206A480151206D08010201E12
:100183000DD21E201F051206BA80031206E6D2A066
:1001930020A014302021C220B2212021051206FC08
:1001A3008015120719801020200DD220202105125E
:1001B30007158003120732D2A120A114302221C2D5
:1001C30022B223202305120736801512075380100D
:1001D30020220DD22220230512074F800312076C21
:1001E300D2A220A214302421C224B2252025051234
:1001F3000770801512078D801020240DD22420252E
:100203000512078980031207A6D2A320A314302660
:1002130021C226B2272027051207AA80151207C775
:10022300801020260DD2262027051207C380031233
:1002330007E0D2A420A414302821C228B2292029FF
:10024300051207E48015120801801020280DD2281A
:100253002029051207FD800312081AD2A520A51430
:10026300302A21C22AB22B202B0512081E80151218
:10027300083B8010202A0DD22A202B051208378034
:1002830003120854D2A620A614302C21C22CB22D5E
:10029300202D0512085880151208758010202C0D8A
:1002A300D22C202D05120871800312088ED2A720AC
:1002B300A714302E21C22EB22F202F0512089280B0
:1002C300151208AF8010202E0DD22E202F051208F4
:1002D300AB80031208C8D2B220B214303421C23426
:1002E300B2352035051208CC80151208EE80102097
:1002F300340DD2342035051208EA800312090CD2DA
:10030300B320B314303621C236B237203705120971
:1003130010801512092D801020360DD23620370596
:100323001209298003120946D2B420B41C7532077E
:1003330012094A12043ED5320675320112094A12D5
:100343000445D2B420B40280EDD2B520B51C753279
:100353000712096212043ED5320675320112096290
:10036300120445D2B520B50280EDD2B620B61C7575
:10037300320712097A12043ED53206753201120988
:100383007A120445D2B620B60280EDD2B720B71C4C
:1003930075320712099512043ED5320675320112E1
:1003A3000995120445D2B720B70280EDE580F535F3
:1003B300A836A935C2D7E899400624FE5010800814
:1003C300C2D7E99824FE50068535361209B0438713
:1003D30001019702003332C0D0C0E0C083C0823035
:1003E3005010C250C2B0D251753300753400D29050
:1003F3008018205115B2900533E5339009CE93F55B
:100403008CD082D083D0E0D0D032B2900534E534A2
:10041300B4FF10C251D290758CFFD082D083D0E04C
:10042300D0D032B40A02D2B0900ACE93F58CD082E7
:10043300D083D0E0D0D032323232327E20DFFEDEC3
:10044300FC227E60DFFEDEFC22D2503099FDC29991
:100453007599B03099FDC2997599403099FDC2994B
:1004630075997F12043E22D2503099FDC299759935
:10047300B03099FDC2997599403099FDC29975992B
:100483000012043E22D2503099FDC2997599B030C2
:1004930099FDC2997599403099FDC29975997F125A
:1004A300043E22D2503099FDC2997599B03099FD1E
:1004B300C2997599403099FDC29975990012043E0D
:1004C30022D2503099FDC2997599B03099FDC299E5
:1004D3007599423099FDC29975997F12043E22D2D3
:1004E300503099FDC2997599B03099FDC2997599AB
:1004F300423099FDC29975990012043E22D25030C0
:1005030099FDC2997599B03099FDC2997599423098
:1005130099FDC29975997F12043E22D2503099FDFC
:10052300C2997599B03099FDC2997599423099FD78
:10053300C29975990012043E22D2503099FDC29996
:100543007599B03099FDC2997599433099FDC29957
:1005530075997F12043E22D2503099FDC299759944
:10056300B03099FDC2997599433099FDC299759937
:100573000012043E22D2503099FDC2997599B030D1
:1005830099FDC2997599433099FDC29975997F1266
:10059300043E22D2503099FDC2997599B03099FD2D
:1005A300C2997599433099FDC29975990012043E19
:1005B30022D2503099FDC2997599B03099FDC299F4
:1005C3007599013099FDC29975997F12043E22D223
:1005D300503099FDC2997599B03099FDC2997599BA
:1005E300013099FDC29975990012043E22D2503010
:1005F30099FDC2997599B03099FDC29975990130E9
:1006030099FDC29975997F12043E22D2503099FD0B
:10061300C2997599B03099FDC2997599013099FDC8
:10062300C29975990012043E22D2503099FDC299A5
:100633007599B03099FDC2997599023099FDC299A7
:1006430075997F12043E22D2503099FDC299759953
:10065300B03099FDC2997599023099FDC299759987
:100663000012043E22D2503099FDC2997599B030E0
:1006730099FDC2997599023099FDC29975997F12B6
:10068300043E22D2503099FDC2997599B03099FD3C
:10069300C2997599023099FDC29975990012043E69
:1006A30022D2503099FDC2997599D03099FDC299E3
:1006B30075997F12043E22D2503099FDC2997599E3
:1006C300D03099FDC29975990012043E22D2503060
:1006D30099FDC2997599D03099FDC29975997F1288
:1006E300043E22D2503099FDC2997599D03099FDBC
:1006F300C29975990012043E22D2503099FDC299D5
:100703007599C03099FDC29975990075300012042E
:100713003E2212043E22D2503099FDC2997599C0EF
:100723003099FDC29975990075300012043E22126A
:10073300043E22D2503099FDC2997599C03099FD7B
:10074300C29975990175300112043E2212043E22AA
:10075300D2503099FDC2997599C03099FDC29975EF
:10076300990175300112043E2212043E22D2503008
:1007730099FDC2997599C03099FDC2997599027511
:10078300300212043E2212043E22D2503099FDC29E
:10079300997599C03099FDC2997599027530021205
:1007A300043E2212043E22D2503099FDC29975991B
:1007B300C03099FDC29975990375300312043E2226
:1007C30012043E22D2503099FDC2997599C03099D6
:1007D300FDC29975990375300312043E2212043E3B
:1007E30022D2503099FDC2997599C03099FDC299B2
:1007F30075990475300412043E2212043E22D2502D
:100803003099FDC2997599C03099FDC299759904C3
:1008130075300412043E2212043E22D2503099FD58
:10082300C2997599C03099FDC299759905753005BE
:1008330012043E2212043E22D2503099FDC2997511
:1008430099C03099FDC29975990575300512043E1A
:100853002212043E22D2503099FDC2997599C030BC
:1008630099FDC29975990675300612043E22120449
:100873003E22D2503099FDC2997599C03099FDC27C
:100883009975990675300612043E2212043E22D24F
:10089300503099FDC2997599C03099FDC2997599E7
:1008A3000775300712043E2212043E22D2503099BB
:1008B300FDC2997599C03099FDC299759907753034
:1008C3000712043E2212043E22D250E53004B4083B
:1008D30001E4F5303099FDC2997599C03099FDC294
:1008E30099F59912043E2212043E22D250E53004B7
:1008F300B40801E4F5303099FDC2997599C0309977
:10090300FDC299F59912043E2212043E22D25030C0
:1009130099FDC2997599C03099FDC2997599017570
:10092300300112043E2212043E22D2503099FDC2FD
:10093300997599C03099FDC2997599007530001267
:10094300043E2212043E22D2503099FDC299759979
:10095300C03099FDC2990531E531547FF59922D212
:10096300503099FDC2997599C03099FDC2991531DE
:10097300E531547FF59922D2503099FDC29975998A
:10098300B03099FDC2997599603099FDC2997599F6
:100993000022D2503099FDC2997599B03099FDC2A9
:1009A300997599613099FDC29975990022D2503099
:1009B30099FDC2997599E03099FDC29975990030F6
:1009C30099FDC299E535C313F59922FFE0FFE0FFD6
:1009D300E0FFE0FFE0FEE1FEE1FEE1FEE1FEE1FD1E
:1009E300E2FDE2FDE2FDE2FDE2FCE3FCE3FCE3FC0D
:1009F300E3FCE3FBE4FBE4FBE4FBE4FBE4FAE5FAFE
:100A0300E5FAE5FAE5FAE5F9E6F9E6F9E6F9E6F9EC
:100A1300E6F8E7F8E7F8E7F8E7F8E7F7E8F7E8F7DD
:100A2300E8F7E8F7E8F6E9F6E9F6E9F6E9F6E9F5CD
:100A3300EAF5EAF5EAF5EAF5EAF4EBF4EBF4EBF4BC
:100A4300EBF4EBF3ECF3ECF3ECF3ECF3ECF2EDF2AD
:100A5300EDF2EDF2EDF2EDF1EEF1EEF1EEF1EEF19C
:100A6300EEF0EFF0EFF0EFF0EFF0EFF0EFF0EFF08C
:100A7300EFF0EFF0EFF0EFF0EFF0EFF0EFF0EFF07B
:100A8300EFF0EFF0EFF0EFF0EFF0EFF0EFF0EFF16A
:100A9300EEF1EEF2EDF2EDF3ECF3ECF4EBF4EBF557
:100AA300EAF5EAF6E9F6E9F7E8F7E8F8E7F8E7F947
:100AB300E6F9E6FAE5FAE5FBE4FBE4FCE3FCE3FD37
:100AC300E2FDE2FEE1FEE1FFE0FFE0E0FFE3FCE642
:100AD300F9E9F6ECF3EFF0F2EDF5EAF8E7FBE4FE03
:100AE300E1FFE0FFE0FFE0FFE0FFE0FEE1FEE1FE0B
:100AF300E1FEE1FEE1FDE2FDE2FDE2FDE2FDE2FCFD
:100B0300E3FCE3FCE3FCE3FCE3FBE4FBE4FBE4FBEB
:100B1300E4FBE4FAE5FAE5FAE5FAE5FAE5F9E6F9DC
:100B2300E6F9E6F9E6F9E6F8E7F8E7F8E7F8E7F8CB
:100B3300E7F7E8F7E8F7E8F7E8F7E8F6E9F6E9F6BC
:100B4300E9F6E9F6E9F5EAF5EAF5EAF5EAF5EAF4AC
:100B5300EBF4EBF4EBF4EBF4EBF3ECF3ECF3ECF39B
:100B6300ECF3ECF2EDF2EDF2EDF2EDF2EDF1EEF18C
:100B7300EEF1EEF1EEF1EEF0EFF0EFF0EFF0EFF07B
:100B8300EFF0EFF0EFF0EFF0EFF0EFF0EFF0EFF169
:100B9300EEF1EEF2EDF2EDF3ECF3ECF4EBF4EBF556
:100BA300EAF5EAF6E9F6E9F7E8F7E8F8E7F8E7F946
:100BB300E6F9E6FAE5FAE5FBE4FBE4FCE3FCE3FD36
:100BC300E2FDE2FEE1FEE1FFE0FFE0204D757A7910
:100BD3006B616E7420342076312E306620323030D3
:100BE300362D31322D3238202863294164616D203E
:100BF300536D69616C656B206A616E6B6F6D757A9D
:100C0300796B616E744077702E706C207777772ED6
:100C1300736D69616C656B2E7072762E706C2057E4
:100C2300737A656C6B6965207072617761207A6194
:100C33007374727A657A6F6E652E204A616B69658B
:100C43006B6F6C7769656B207A6173746F736F7701
:100C5300616E6961206B6F6D657263796A6E652081
:100C63006B6F6475206E6965646F7A776F6C6F6EF6
:100C7300652E20416C6C205269676874732052653D
:100C83007365727665642E204672656520666F72A1
:100C9300206E6F6E20636F6D6D65726369616C208A
:060CA3006F6E6C792E203B
:00000001FF
